:020000020000FC
:1000000021C0189518951895CFB6D39429F4750189
:1000100075B5786475BD93BCFD1409F4E3BC7F2D00
:10002000739529F07D1519F475B5777B75BDCFBE35
:100030001895C09A8895C09808B702FFFACF04E0D7
:1000400008BF0895882499249A9404E00EBF0FE510
:100050000DBF00E409BF09E605BD02EA0FBD09E1D5
:100060000EBD97BC96BC482C582C692C0FE107BBE1
:1000700000E805BF7894DDDF6A942BD0439411D05B
:100080004914C9F7D6DF4A940CD0539416D05914AA
:10009000C9F7CFDF5A9411D063941BD06914C9F704
:1000A000EACFE42D21D01BBD0ABD0FB5442011F0CD
:1000B000006801C00F770FBD0895E52D15D019BD5B
:1000C00008BD0FB5552011F0006201C00F7D0FBDB6
:1000D0000895E62D09D0580105B5662011F000629B
:1000E00001C00F7D05BD0895FF27EE0FFF1FE850EB
:1000F000FF4F0591159108950000000001000200D6
:100100000300040005000700080009000A000C00B5
:100110000D000F001000120013001500160018004B
:100120001A001C001E0020002200240026002800C7
:100130002A002C002F0031003400360039003C002A
:100140003F004100440048004B004E005100550064
:1001500059005C006000640068006C00710075006C
:100160007A007E00830088008D00920098009E0037
:10017000A300A900AF00B600BC00C300CA00D100B4
:10018000D800E000E800F000F800010109011301C7
:100190001C0125012F013A0144014F015A0166015A
:1001A00071017E018A019701A401B201C001CF0152
:1001B000DE01ED01FD010E021F0230024202540277
:1001C00068027B028F02A402BA02D002E702FE029A
:1001D00016032F03490363037E039B03B703D50371
:1001E000F40314043404560478049C04C004E604A4
:1001F0000D0535055F058905B505E20511064106C2
:100200007206A506D9060F0747078007BC07F8073F
:1002100037087808BA08FF0845098E09D909260A5F
:10022000760AC80A1C0B730BCD0B290C880CEA0C40
:100230004F0DB70D220E910E020F770FF00F6C10BD
:10024000EC107011F81184121513A9134214E01464
:1002500083152A16D71688173F18FC18BE19861A58
:10026000551B291C041DE61DCE1EBD1FB420B22146
:10027000B722C523DB24F92520274F288829CA2A3D
:10028000172C6D2DCD2E3830AE313033BD3456366F
:10029000FB37AD396C3B393D143FFD40F442FB4424
:1002A00012473949704BB94D13508052FF54915742
:1002B000385AF35CC35FA962A565B868E36B276F22
:1002C0008472FB758D793A7D0481EB84F088148DFE
:1002D0005991BE95469AF09EBFA3B2A8CCAD0EB37D
:1002E00078B80CBECBC3B7C9D1CF19D693DC3EE3E7
:0802F0001DEA31F17CF8FFFF6B
:00000001FF
